:020000040000FA
:04000000CD303A289D
:08000800A000030EA100831209
:100010008B1C32288B1031181428B11C3228643004
:10002000010203183128182800001628172818285C
:1000300019281A281B281C281D281E281F283110A3
:10004000B114A810031005190314AA0DA90DA80DC9
:10005000B00B322831152A08AF002908AE00280855
:10006000AD00B11081010B11210E8300A00E200EF6
:02007000090085
:0C007400203084008001840A80300402E7
:10008000031C3C281230B000F72183160C30850584
:1000900087018312850187010730990000309A009B
:1000A000103083168E008312603083168F00831207
:1000B0000030831691009F008312C83083168100A0
:1000C000831231309000003083168C008312103080
:1000D0008B00BC1B6D28851D2623092381018E0101
:1000E0008F010B118B100B108C018B178520311990
:1000F0009B20B30B8328031085190314B90DF0302E
:100100003902031953216C23762864003118080042
:100110000B1D08000B11B11031141230B000051D79
:1001200096283214831601138312080032108316A6
:1001300001178312080031110130B7008B132030F2
:10014000370783169B001C141A088312A400A5000D
:10015000C030A5061030370783169B001C141A0800
:100160008312A3000030370783169B001C141A0863
:100170008312A2008B17321CC32822090339A20064
:10018000A309A409A50922082D02031D4D2923084E
:100190002E02031D4D2924082F02031D4D29013075
:1001A0003702031DD8283D18D8283D143E141922C3
:1001B00002303702031DE128BD18E128BD143E14AA
:1001C000282203303702031DEA283D19EA283D158D
:1001D0003E14342204303702031DF328BD19F328DE
:1001E000BD153E14402205303702031DFC283D1A80
:1001F000FC283D163E144C2206303702031D05290B
:10020000BD1A0529BD163E14582207303702031DBA
:100210000E293D1B0E293D173E1467220830370278
:10022000031D1729BD1B1729BD173E14762209305F
:100230003702031D20295E1820295E143E148122F6
:100240000A303702031D2929DE182929DE143E143D
:100250008C220B303702031D32295E1932295E15BC
:100260003E1497220C303702031D3B29DE193B292F
:10027000DE153E14A2220D303702031D44295E1AFA
:1002800044295E163E14AD220E303702031D4D295F
:10029000DE1A4D29DE163E14B822B70A0F30370297
:1002A000031808009E280130B600B300B400B50062
:1002B000B70085018701B1138520B30BA329031073
:1002C00085190314B90DF03039020319CA29B40B8A
:1002D000A329013037020319C32202303702031960
:1002E000C822033037020319CD2204303702031924
:1002F000D222053037020319D722063037020319FC
:10030000DC22073037020319E122083037020319D3
:10031000E622093037020319EB220A3037020319AB
:10032000F0220B3037020319F5220C303702031983
:10033000FA220D3037020319FF220E30370203195B
:1003400004239630B400311D5C293111321CAD29D3
:100350002D090339AD00AE09AF092F1CB1132F1CB5
:100360005C29B11B5C292E185C29B1178B13203036
:100370003707BB002F08BA00E22110303707BB0057
:100380002E08BA00E22100303707BB002D08BA0062
:10039000E2218B1785018701B70AB6010F303702BA
:1003A000031C5C29092308003E1C08003E10103085
:1003B000BB003D08BA00E2213030BB005E08BA0045
:1003C000E22108008B133A0883161C159A00831249
:1003D0003B0883169B0055309D00AA309D009C145D
:1003E00064009C18F0291C1183128B1708008316D7
:1003F00000309B001C141A088312BC0083161030B6
:100400009B001C141A088312BD00831630309B0019
:100410001C141A088312DE00FF30C800CA15CB1561
:10042000CC15CD15CE15CF15D015D115D215D315A8
:1004300008008130BD05FF30DE054130C405C00035
:100440000030C200C600BC185F14BC18DF140800DE
:100450008230BD05FF30DE058030C405C0000030AD
:10046000C200C6005F1008008430BD05FF30DE0505
:100470004230C405C0004030C200C6005F10080012
:100480008830BD05FF30DE054630C405C000403071
:10049000C200C6005F1008009030BD05FF30DE05C9
:1004A0008A30C405C0008030C200C6005F1008005A
:1004B000A030BD05FF30DE055130C405C00010304E
:1004C000C200C600BC185F14BC18DF140800C0309E
:1004D000BD05FF30DE057130C405C0000030C2002C
:1004E000C600BC185F14BC18DF140800FF30BD053F
:1004F000C030DE054030C505C1000030C300C70074
:1005000008007F30BD05C130DE058030C505C10063
:100510000030C300C70008007F30BD05C230DE05D3
:100520004030C505C1004030C300C70008007F301F
:10053000BD05C430DE054030C505C1004030C300F4
:10054000C70008007F30BD05C830DE058030C50516
:10055000C1008030C300C70008007F30BD05D03027
:10056000DE054030C505C1000030C300C7000800EB
:100570007F30BD05E030DE054030C505C1000030EC
:10058000C300C70008001030850600308706080049
:100590003330850606308706080020308506003097
:1005A00087060800213085060030870608002230C3
:1005B0008506003087060800103085060230870661
:1005C00008001030850606308706080000308506D2
:1005D00010308706080000308506083087060800BE
:1005E0000030850610308706080000308506103080
:1005F00087060800003085060830870608000030AE
:100600008506103087060800003085061030870602
:1006100008003D181922BD1828223D193422BD19A1
:1006200040223D1A4C22BD1A58223D1B6722BD1B99
:1006300076225E188122DE188C225E199722DE193E
:10064000A2225E1AAD22DE1AB8220800B601B3015A
:10065000B4013C1C2E2BBC01BC14302BBC013C143F
:100660003C08B6006400342B352B362B372B382B47
:10067000FF30B41B8500B41F8501B30B322BB40BC4
:10068000322B0310B60CB608031D322B0030BB0012
:100690003C08BA00E221080005125C180516DC1CB3
:1006A0008512DC1885165C1D05105C190514DC1D0F
:1006B0008510DC1985145C1E87105C1A8714DC1EFB
:1006C0000711DC1A07155C1F07105C1B0714DC1FE1
:1006D0008712DC1B871608008F08031908008F019A
:1006E00078308E00C80F9A2DC80A441C9C2B461CDB
:1006F0008D2BCA1C7E2BCA014A15AA2B4A1D832B9F
:10070000CA01CA15AA2BCA1D882BCA014A16AA2BD0
:100710004A1EAA2BCA01CA14AA2B4A1D922BCA012F
:100720004A16AA2BCA1D972BCA014A16AA2B4A1E83
:10073000AA2BCA01CA14AA2BCA1CA12BCA014A158A
:10074000AA2B4A1DA62BCA01CA15AA2B4A1EAA2BE0
:10075000CA014A15C41CD12BC61CC22BCB1CB32BFF
:10076000CB014B15DF2B4B1DB82BCB01CB15DF2B52
:10077000CB1DBD2BCB014B16DF2B4B1EDF2BCB0133
:10078000CB14DF2B4B1DC72BCB014B16DF2BCB1D07
:10079000CC2BCB014B16DF2B4B1EDF2BCB01CB140D
:1007A000DF2BCB1CD62BCB014B15DF2B4B1DDB2BB3
:1007B000CB01CB15DF2B4B1EDF2BCB014B15441D83
:1007C000062C461DF72BCC1CE82BCC014C15142C09
:1007D0004C1DED2BCC01CC15142CCC1DF22BCC01D7
:1007E0004C16142C4C1E142CCC01CC14142C4C1D67
:1007F000FC2BCC014C16142CCC1D012CCC014C161E
:10080000142C4C1E142CCC01CC14142CCC1C0B2CF2
:10081000CC014C15142C4C1D102CCC01CC15142CD7
:100820004C1E142CCC014C15C41D3C2CC61D2D2C6B
:10083000CD1C1E2CCD014D155F134A2C4D1D232CB4
:10084000CD01CD154A2CCD1D282CCD014D164A2C9D
:100850004D1E4A2CCD01CD144A2C4D1D322CCD01FC
:100860004D164A2CCD1D372CCD014D164A2C4D1E50
:100870004A2CCD01CD144A2CCD1C412CCD014D1557
:100880004A2C4D1D462CCD01CD154A2C4D1E4A2C0F
:10089000CD014D155F1B732C441E732C461E642C1A
:1008A000CE1C552CCE014E15812C4E1D5A2CCE013E
:1008B000CE15812CCE1D5F2CCE014E16812C4E1EE6
:1008C000812CCE01CE14812C4E1D692CCE014E16EA
:1008D000812CCE1D6E2CCE014E16812C4E1E812CED
:1008E000CE01CE14812CCE1C782CCE014E15812C3D
:1008F0004E1D7D2CCE01CE15812C4E1E812CCE019D
:100900004E15C41EA82CC61E992CCF1C8A2CCF01B4
:100910004F15B62C4F1D8F2CCF01CF15B62CCF1DE8
:10092000942CCF014F16B62C4F1EB62CCF01CF14EE
:10093000B62C4F1D9E2CCF014F16B62CCF1DA32CCD
:10094000CF014F16B62C4F1EB62CCF01CF14B62CAC
:10095000CF1CAD2CCF014F15B62C4F1DB22CCF01A3
:10096000CF15B62C4F1EB62CCF014F15441FDD2CD2
:10097000461FCE2CD01CBF2CD0015015EB2C501D87
:10098000C42CD001D015EB2CD01DC92CD001501691
:10099000EB2C501EEB2CD001D014EB2C501DD32C83
:1009A000D0015016EB2CD01DD82CD0015016EB2CBA
:1009B000501EEB2CD001D014EB2CD01CE22CD0011B
:1009C0005015EB2C501DE72CD001D015EB2C501EF0
:1009D000EB2CD0015015C41F122DC61F032DD11CA6
:1009E000F42CD1015115202D511DF92CD101D11517
:1009F000202DD11DFE2CD1015116202D511E202D50
:100A0000D101D114202D511D082DD1015116202DB9
:100A1000D11D0D2DD1015116202D511E202DD1019A
:100A2000D114202DD11C172DD1015115202D511D70
:100A30001C2DD101D115202D511E202DD101511574
:100A4000DF184A2D451F4A2D471F3B2DD21C2C2D48
:100A5000D2015215DF13582D521D312DD201D2155E
:100A6000582DD21D362DD2015216582D521E582DFA
:100A7000D201D214582D521D402DD2015216582D9C
:100A8000D21D452DD2015216582D521E582DD2017D
:100A9000D214582DD21C4F2DD2015215582D521D53
:100AA000542DD201D215582D521E582DD201521557
:100AB000DF18832DDF1B832DC51F832DC71F742DCA
:100AC000D31C652DD3015315912D531D6A2DD301D0
:100AD000D315912DD31D6F2DD3015316912D531E78
:100AE000912DD301D314912D531D792DD30153167C
:100AF000912DD31D7E2DD3015316912D531E912D73
:100B0000D301D314912DD31C882DD3015315912DCE
:100B1000531D8D2DD301D315912D531E912DD3012E
:100B20005315D4214008C4004108C5005F18DF14E4
:100B30005F1CDF104808C9000C304A05031D051270
:100B40000C304B05031D85120C304C05031D0510A0
:100B50000C304D05031D85100C304E05031D87100C
:100B60000C304F05031D07110C305005031D0710F5
:100B70000C305105031D87120C305205031D07125E
:100B80000C305305031D871149080E020318F42D7C
:100B900012304A05031D051612304B05031D85163C
:100BA00012304C05031D051412304D05031D85142C
:100BB00012304E05031D871412304F05031D071513
:100BC00012305005031D071412305105031D8716FE
:100BD00012305205031D071612305305031D8715E9
:100BE000FF304802031908008F08031D0800852004
:100BF00049080E02031CF42D18304A05031D051286
:100C000006304A05031D051618304B05031D8512D5
:100C100006304B05031D851618304C05031D0510C5
:100C200006304C05031D051418304D05031D8510B5
:100C300006304D05031D851418304E05031D871021
:100C400006304E05031D871418304F05031D07118C
:100C500006304F05031D071518305005031D0710FA
:100C600006305005031D071418305105031D871267
:100C700006305105031D871618305205031D071253
:100C800006305205031D071618305305031D871142
:0A0C900006305305031D8715080008
:084000000500030005000500A6
:02400E00CC33B1
:10420000010003000300030003000200020002009B
:104210000200000000000000000003000300FF0097
:10422000810000000000000000000000000000000D
:104230000000C000C000C000C000C000C000FF00FF
:10424000FF00C300F300CF00FF00C300F300CF0066
:10425000FF00C300F300CF00FF00C300F300FF0026
:104260000000FF00FF00FF00FF00FF00FF00FF0055
:10427000FF00FF00FF00FF00FF00FF00FF00FF0046
:10428000FF00FF00FF00FF00FF00FF00FF00FF0036
:10429000FF00FF00FF00FF00FF00FF00FF00FF0026
:1042A000FF00FF00FF00FF00FF00FF00FF00FF0016
:1042B000FF00FF00FF00FF00FF00FF00FF00FF0006
:1042C000FF00FF00FF00FF00FF00FF00FF00FF00F6
:1042D000FF00FF00FF00FF00FF00FF00FF00FF00E6
:1042E000FF00FF00FF00FF00FF00FF00FF00FF00D6
:1042F000FF00FF00FF00FF00FF00FF00FF00AA001B
:00000001FF
